:0300000002045F98
:0C045F00787FE4F6D8FD7581370204A612
:0D06CB000B233F065B4F666D7D077F6F3987
:1005D600E4FBFAC2B6EF70047D0D80027D0FE4FCE9
:1005E600C2A4ED30E304D2948002C294D2A4ED25D5
:1005F600E0FD0CBC04EAD294C2A4E4FCEB25E0FBCB
:10060600EA33FAD2A4C2A43094054303018003530B
:0E06160003FE0CBC0CE6D2B6EA540FFEAF0396
:0106240022B3
:10062500E4FFE4FE742E2FF8E6FD30E704D2B78030
:1006350002C2B7D2A4742E2FF8ED25E0F6C2A40E9F
:0B064500BE08E10FBF04DBD2A5C2A578
:010650002287
:10056C001203CE8E208F217C037DE812036B742343
:10057C002FF8E6F52EAE20AF217C037DE812036B3D
:10058C008C208D21AE20AF217C007D6412036B7416
:10059C00232FF8E6F52FAE20AF217C007D641203EB
:1005AC006B8C208D21AE20AF217C007D0A12036B59
:1005BC0074232FF8E6F530AE20AF217C007D0A12B3
:0A05CC00036B74232DF8E6F53122CD
:10067300051BE51B7002051AD3940AE51A648094DE
:0F06830080400BE4F51AF51B12056C12062522B8
:10069200051DE51D7002051CD39432E51C6480948F
:0E06A20080400AE4F51CF51DA292B39292224C
:1004EB0085181E85191F85161885171985141685ED
:1004FB001517851214851315851012851113850E8A
:10050B0010850F11850C0E850D0F850A0C850B0DB3
:10051B0085080A85090B7F011205D68E088F09E520
:10052B0009250BCFE508350ACF250DCF350CCF2587
:10053B000FCF350ECF2511CF3510CF2513CF351259
:10054B00CF2515CF3514CF2517CF3516CF2519CF7E
:10055B003518CF251FCF351EFE7C007D0A12036B8D
:01056B00226D
:1003CE00E4F537F536F535F534F532F533AB37AAB6
:1003DE0036A935A834C000C001C002C0037F011287
:1003EE0005D6AC06AD07EC1202B1D003D002D00197
:1003FE00D0001200158F378E368D358C340533E5CF
:10040E003370020532C3E5326480948140BFAF374A
:10041E00AE36AD35AC34E4FBFA7980784312020F78
:10042E008F378E368D358C347B0A7AD77923783C8C
:10043E001201068F378E368D358C34E4FFFE7D5CCF
:10044E007C43AB37AA36A935A8341201061202EA4C
:01045E00227B
:100651001204EBAC06AD07EC1202B17B017A4D79C5
:1006610004783D1201067BB67AF3797178C11200E4
:02067100152250
:03000B000206D911
:0906D900758CD8758AF0052232F7
:1006B000D2AFD2A9438901D28CE4F522E52260FCB5
:0B06C000E4F52212067312069280F18E
:10000E00020356E86480F8E933E83360110460F0C7
:10001E00ED33EC337009E8FCE9FDEAFEEBFF220458
:10002E0060DED3EB9FEA9EE99DE8C2E78CF0C2F753
:10003E0095F0400CE8CCF8E9CDF9EACEFAEBCFFB1F
:10004E0012032185D0F05804700320D5B3E8047054
:10005E00075002B2D502036092D5EC0460F7E4CCEF
:10006E00C0E0C398F8603B94186008400DD0E0FBE8
:10007E00020338E4FBFAC9FC8028E830E406E4C940
:10008E00FBE4CAFCE830E305E4C9CACBFCE854073C
:10009E006010F8C3E913F9EA13FAEB13FBEC13FC47
:1000AE00D8F130F52FC3E49CFCEF9BFFEE9AFEEDEA
:1000BE0099FDD0E0FBEF4E4D4C701222DB03020394
:1000CE005DEC2CFCEF33FFEE33FEED33FDED30E750
:1000DE00EB020338EF2BFFEE3AFEED39FDD0E0FBDD
:1000EE0050130BBB0003020360ED13FDEE13FEEF86
:0800FE0013FFEC13FC020338B0
:10010600EC4D6011E8497017ED33EC3304600DE4F3
:10011600FCFFFEFD22E933E8330470F802035612B1
:10012600032158046009E4CC2481500628500902B2
:10013600036028400302035DC0E0EB4A7044B980C7
:1001460006D0E0FB02034CEF4E701CBD8008EBFFAF
:10015600EAFEE9FD80EBE98DF0A4FEE5F00201EF91
:10016600E9CDF9EAFEEBFFEF89F0A4FCE5F0CE89D4
:10017600F0A42EFFE435F0CD89F0A42DFEE435F091
:100186008067EF4E7005BD80D780C3EF8BF0A4ACBF
:10019600F0EE8BF0A42CFCE435F0F8EF8AF0A42CFA
:1001A600E5F038FCE433CB8DF0A42CFCE5F03BF80D
:1001B600EE8AF0A42CFCE5F038F8E433CF89F0A4FD
:1001C6002CFCE5F038CF3400CE89F0A42FFFE5F003
:1001D6003EFEE433C98DF0A42EFEE5F039CD8AF05B
:1001E600A42FFFE5F03EFEE43DFD33D0E0FB5007D3
:1001F6000BBB000F020360EC2CFCEF33FFEE33FE6B
:06020600ED33FD02033898
:10020C00020360EC5D046005E859047003020356B8
:10021C00120321580460F6EC4860F2EC7004FDFE09
:10022C00FF22C860DB2481C85009C39860025006C5
:10023C0002035D9850CAF582E9294B4A7005AB82DE
:10024C0002034C75F0007C1A7880C3EF9BEE9AED9C
:10025C0099400DC3EF9BFFEE9AFEED99FDE842F03D
:10026C00DC23ACF0D0E0FFD0E0FED0E0FDAB822090
:10027C00E7101BEB60BAEC2CFCEF33FFEE33FEED1A
:10028C0033FD020338E803F830E705C0F075F000E1
:10029C00EF2FFFEE33FEED33FD40B830E7C280AAFE
:1002AC0075F020800E75F010800575F0087D007ECD
:1002BC00007F003392D530D5031203C0EC334010CD
:1002CC00EF33FFEE33FEED33FDEC33FCD5F0ED22D6
:0E02DC00E5F0247EA2D513CC92E7CDCEFF2212
:1002EA00EDD2E7CD33EC3392D524814006E4FFFE0C
:1002FA00FDFC22FCE4CFCECDCC24E0501174FF806B
:10030A00EDC3CC13CCCD13CDCE13CECF13CF047007
:07031A00F030D5DE0203C044
:10032100E9D2E7C933E833F892D5EDD2E7CD33EC22
:0703310033FC5002B2D5229B
:10033800EC30E7100FBF000C0EBE00080DBD000426
:100348000BEB6014A2D5EB13FCED92E7FD2274FFD2
:10035800FCFDFEFF22E480F8A2D574FF13FC7D802B
:03036800E480EF3F
:10046B000206B0E493A3F8E493A34003F68001F2F1
:10047B0008DFF48029E493A3F85407240CC8C33392
:10048B00C4540F4420C8834004F456800146F6DF61
:10049B00E4800B01020408102040809006CBE47E20
:1004AB00019360BCA3FF543F30E509541FFEE49356
:1004BB00A360010ECF54C025E060A840B8E493A31D
:1004CB00FAE493A3F8E493A3C8C582C8CAC583CA48
:1004DB00F0A3C8C582C8CAC583CADFE9DEE780BE00
:0106D8000021
:10036B00BC000BBE0029EF8DF084FFADF022E4CC76
:10037B00F875F008EF2FFFEE33FEEC33FCEE9DEC3F
:10038B00984005FCEE9DFE0FD5F0E9E4CEFD22ED85
:10039B00F8F5F0EE8420D21CFEADF075F008EF2FCF
:1003AB00FFED33FD4007985006D5F0F222C398FDC0
:0503BB000FD5F0EA225D
:0E03C000C3E49FFFE49EFEE49DFDE49CFC224E
:00000001FF
